:030000000210E308
:03000B000200A54B
:03002B000202AE20
:03005B0002040C90
:030073000203E69F
:1000800002030406080C10182030406080040608A3
:100090000C10182030406080A0C00D0D0405060D26
:1000A0000503030302C2AFC0D0C0E020620C206889
:1000B00002419D306602415DE47385258AC262E596
:1000C00025F4700221242068022111207210758B02
:1000D00000D0E0D0D0D292D291D290D2AF32D29290
:1000E000D291D2907406D5E0FDE53C1420E21520B3
:1000F000E10D207D02D295307D02D293020121D202
:1001000094020121207D02D293307D02D29502011A
:1001100021758B00D0E0D0D0D292D291D290D2AFC4
:1001200032758B00D0E0D0D0D2AF32419DE5256052
:100130000A207D02C292307D02C290D291419DE59B
:10014000256002C291207D02D290307D02D2924180
:100150009DE525600A207D02C290307D02C292207A
:100160007D02D292307D02D290419D207D02C293C9
:10017000307D02C295207D02C295307D02C293740B
:1001800006D5E0FDE525600A207D02C292307D02A1
:10019000C290D291419D207D02C293307D02C295D2
:1001A000C2947406D5E0FDE525600A207D02C29266
:1001B000307D02C290D291419DC294207D02C293B3
:1001C000307D02C2957406D5E0FDE5256002C2913E
:1001D000207D02D290307D02D292419DC294207D3A
:1001E00002C295307D02C2937406D5E0FDE525601C
:1001F00002C291207D02D290307D02D292419D2098
:100200007D02C295307D02C293C2947406D5E0FD92
:10021000E525600A207D02C290307D02C292207DD9
:1002200002D292307D02D290419D207D02C2953053
:100230007D02C293207D02C293307D02C295740676
:10024000D5E0FDE525600A207D02C290307D02C226
:1002500092207D02D292307D02D290419D30723D3B
:10026000E53C20E21A20E129207D02C293307D0284
:10027000C295207D02C295307D02C29302029D206C
:10028000E1E6207D02C293307D02C295C294020253
:100290009DC294207D02C295307D02C293E525F473
:1002A000F58A758B00D262D0E0D0D0D2AF32C2AF27
:1002B000C2AD53E6EFC0D0C0E0D2D3D2AFC2CEE5DC
:1002C0002960072074461529610C78007900E580C3
:1002D000307E01F430E40278FF53DACF207E03430E
:1002E000DA20307E0343DA10C2D8C271E580307E56
:1002F00001F430E40279FFC3E89970CE30610375F0
:1003000029182074037529188859D270E52A6004C9
:10031000152A611C20740543DA01C2D820700261DD
:1003200083A859206102C2702074367982B70431E3
:10033000C3E894F0400374F0F8E8C4540F28F87947
:1003400084B703026161C313C3138721200802C36A
:1003500013200A06C3C898F8616128F8500374FF97
:10036000F88822306915E5222408F5225003752209
:10037000FFC3E522955E4003855E227882B60418AD
:10038000852224A824C3E524955E4002A85EC3E824
:1003900095604002A8608825C3E52594404002D2BC
:1003A0006420CF0CD0E0D0D0C2D343E610D2AD321F
:1003B000C2CF7801E52960053074021529C3E559DB
:1003C00094014005755C0061DA755D00756400E5B7
:1003D0005C2401F55C5003755CFFD0E0D0D0C2D343
:1003E00043E610D2AD32C0D0C0E0C2AF53917F53CC
:1003F000E67FC260759100C3E49550F594E4955191
:10040000F595759104D0E0D0D0D2AF32C2AF53E6AB
:10041000EFC2ADC0D0C0E0C0F0D2D3D2AFA8FBA92C
:10042000FCC2D8307102817353DACF207E0343DAE5
:1004300010307E0343DA20D271E580307E01F42053
:10044000E402814A88268927C1AF53DACF207E0390
:1004500043DA20307E0343DA10C2D8C2713074020E
:10046000C19B7800E580307E01F430E402C19B88B6
:0F04700059C18253DACF207E0343DA20307E0356
:10047F0043DA10C271206102A14353DACF207E0309
:10048F0043DA10307E0343DA20C2D8D27188548900
:10049F0055C3E89552F8E99553F9E4FB7E027A00CB
:1004AF00C3E8948CE994005005755800A133C3E854
:1004BF0094C8E994005008E4D2E4FB7A0AA110C36F
:1004CF00E89468E994015008E4D2E3FB7A0FA11095
:1004DF00C3E894D0E994025008E4D2E2FB7A1EA15B
:1004EF0010C3E894A0E994055008E4D2E1FB7A3CEC
:1004FF00A110C3E89498E994085008E4D2E0FB7A7D
:10050F00787E00C3E89556FCE99557FD30E708EC77
:10051F00F42401FCEDF4FD755800C3EC9AED9E50E8
:10052F000375580188568957A854A955885289537D
:10053F007802C182C3E89526F8E99527F9307C0245
:10054F00C166307B02C166307A02C15F207502A19D
:10055F0066E9FDE8FCA185E9C313F9E813F83079E2
:10056F0002C15FE9C313F9E813F8307802C15FE9FC
:10057F00C313FDE813FC206126C3EC941CED940219
:10058F004002A19CED7018C3EC94C850120528C30B
:10059F00E528940A5002C19B755900D270C19BE5A2
:1005AF0028600215287400207F0B7888E67896B4AF
:1005BF000302789EE624FAFEE43400FFC3EC9EFCAF
:1005CF00ED9FFD92087888E6B40327A20850092012
:1005DF007D20C2AFD27DA1EE307D17C2AFC27DD2DA
:1005EF0092D291D290C293C294C295206902D26BDB
:1005FF00D2AFA2085017E6B4030DECF42401FCEDC2
:10060F00F43400FD02061C78007900C1667888E694
:10061F00B40315EC33FCED33FDC3EC940AFCED94FD
:10062F0000FD50047C007D00C3EC94FFED9400406E
:10063F000678FF7900C166EC856FF0A4C5F0A2F7CC
:10064F0033F87900400302068278FF7900020682B0
:10065F00E9C313F9E813F8307C0EE9600278FFC3A1
:10066F00E81338F8E43400F9C3E894FFE994004044
:10067F000278FF8859D270206102C19B741FF45514
:10068F002F4BF52FC274E42B7002D27475291830DA
:10069F00740375290A306102C1AF20740353DAFE67
:1006AF00752A06307403752A0AD0F0D0E0D0D0C274
:1006BF00D3D2AD43E6103279010206E47903020684
:1006CF00E4790A0206E4791E0206E479640206E47C
:1006DF0079C80206E47817E4D5E0FDD8FAD9F622F6
:1006EF007A147B7802070B7A107B8C02070B7A0D3A
:1006FF007BB402070B7A0B7BC802070BAC25752561
:10070F00017902B27DE4C294D5E0FDE5256002C215
:10071F0091D5E0FDD291D5E0FDD294D5E0FDE52550
:10072F00600A207D02C292307D02C290E570D5E052
:10073F00FD207D02D292307D02D2907496D5E0FDDD
:10074F00D9C1EAF8D5E0FDD8FBDBB1C2948C2522E4
:10075F00C37C007D0075F00005F0EA33FAEB33FB44
:10076F0050F6EB13FBEA13FAC3E9FFE8FEE89AF839
:10077F00E99BF95004EFF9EEF8B3EC33FCED33FDE0
:10078F00D5F0DFEDF9ECF822E889F08A20D2D4F821
:10079F00A9F07B0030F70B7BFFF42401F8E9F43468
:1007AF0000F9E88520F0A4ADF0F8E98520F0A4AFBA
:1007BF00F0FEED2EF974003FFA7C04C3EA13FAE958
:1007CF0013F9E813F8DCF48BF030F70AE8F424019E
:1007DF00F8E9F43400F9E889F0C2D4F8A9F02278E6
:1007EF0082B6040302084BC3E55994014003020883
:1007FF0013852224E4F53EF53FF540F541F542F52A
:10080F004702084B7882E6FC754701E522F523780D
:10081F003879C7AA3AAB3BC3EB13FBEA13FAEC14D4
:10082F006013C3EB13FBEA13FAEC14146007C3EB6A
:10083F0013FBEA13FA12075F883E893F22E54760F0
:10084F0034C3E53E9523F8E53F9400F9500CC3E817
:10085F009480E994FF4016020880C3E8947FE994DE
:0F086F00005003020880787F79000208807880AB
:10087E0079FF8843894422E5476058E5432540F8CF
:10088E00E5443541F9854420E4300701F43542FA58
:10089E0030E709C3EA94F040150208C2C3EA940F88
:1008AE0050030208C278FF79FF7A0F0208C278005F
:1008BE0079007AF0C3E524955E5006E524600901BF
:1008CE00DBE54420E70D01DBE54430E7068840898F
:1008DE00418A4222E547700302094678A1E6FAC32F
:1008EE00E54333F8E54433F9120797E930E70BC3D4
:1008FE00E89480E994FF4013211DC3E8947FE994A6
:10090E00005002211D787F7900211D788079FFE843
:10091E0020E715C3E52398F84009C3E89401400386
:10092E000209447801020944E8F424012523F84021
:10093E000302094478FF884522E54770030209A99E
:10094E0078A2E6FAA841A942120797E930E70CC34C
:10095E00E89401E994FF4016020980C3E894FFE988
:10096E009400500302098078FF7900020980780113
:10097E0079FFE920E715C3E54598F84009C3E894E7
:10098E000140030209A778000209A7E8F424012513
:10099E0045F840030209A778FF88242278FFC26435
:1009AE00E52D5406702FD264C3E53B940A4009C36B
:1009BE00E52594405002C264E53B601974FF853B07
:1009CE00F0848537F0A4F8C5F0600278FFC3E8958F
:1009DE00615002A8618860227883E6F520120F0428
:1009EE0075E8901206C675E890E5E820ECFBA8BD08
:1009FE00A9BE120F9A756BAF756C00C3740013FD10
:100A0E0074AF13FC74AF2CFC74003DFDECFAEDFBDF
:100A1E00C3E89AE99B4014E56B24AFF56BE56C34A3
:100A2E0000F56CEA2CFAEB3DFB80E5AE6BAF6CC3C8
:100A3E00E56C13F9E56B13F8C3E913F9E813F8E560
:100A4E006B28F569E56C39F56A7A03C3E913F9E8A1
:100A5E0013F8DAF7AA201A7009756B00756C00028C
:100A6E000A801AEA6008EE28FEEF39FFDAF88E6B7C
:100A7E008F6C2275E890227883E6FFE5E820ECF78C
:100A8E00A8BDA9BE056DC3E56D94084052756D00F5
:100A9E00E9FA79A0E76044EA7007E56E601B020A86
:100AAE00BBC3E8956E6010E56E5006600C14020A2A
:100ABE00C70460F9020AC7E56EF56EC39458401B71
:100ACE00755EC0C394044013755E80C39404400BDE
:100ADE00755E40C394044003755E0075BB0322EF40
:100AEE00C39401601BC3E894FFE994035012C3E85A
:100AFE00956BE9956C5009E55E601A155E020B2345
:100B0E00E55EF46010055E7888E6B40308E55E24C1
:100B1E00044002F55EA85EC3E524985002A824C3E3
:100B2E00E8955F400AA85FE55FF46003855F5E7934
:100B3E0082B70402614EC3E895604002A860882522
:100B4E00E56DB4070375BB1022743279A387F0A448
:100B5E00C5F0A2F733F8C3E8955E4002A85E88227E
:100B6E0088248825886122753A00753B7F2275C8D6
:100B7E0020A8CCA9CD75C824AA38AB3988388939B4
:100B8E00C3E89AF8E99BF9AA3AAB3BAC3AAD3B7E87
:100B9E00047F02C3EB940440021E1FC3EB94084073
:100BAE00021E1FC3ED13FDEC13FCDEF7C3EA9CFA25
:100BBE00EB9DFBEF6009C3E913F9E813F8DFF7EAE1
:100BCE0028FAEB39FB8A3A8B3B400122753AFF75C6
:100BDE003BFF2230600261E1854C50854D51D26061
:100BEE0043E680227892E6FFC3E535948240010FFA
:100BFE00C3E53594A040010FC3EF940640027F0574
:100C0E007E021E3072010EC3E53B940350060E0E9B
:100C1E003072010EC3E53B940250060E0E30720187
:100C2E000EA93BA83A7A04C3E913F9E813F8DAF7E8
:100C3E00C3E89EF8E99400F94009C3E89402E994E8
:100C4E000050047802E4F9E9FBE8FAC3E913FDE881
:100C5E0013FC884C894DC3EF94036037EF20E00DF1
:0F0C6E00E82CF8E93DF9ECFAEDFB020C8EE828D2
:100C7D00F8E939F9C3E89402F8E99400F97A02E445
:100C8D00FBC3EF9403400D8A4E8B4F884889498CE6
:100C9D004A8D4B22884E894F8A488B498C4A8D4B01
:100CAD002230600281AED26043E680E52D540660AD
:100CBD0027A83AA93BE53494085006E820E002A99C
:100CCD004D759100C3E498F594E499F595759104EB
:100CDD00D26053917F43E68022D265753D00752029
:100CED0000020CF9D265753D00752040E52D5406C6
:100CFD006002C265D2AF206005E53D60012278013A
:100D0D007A02C3E53B940540027802C3E53B940AA1
:100D1D0040027803C3E53B940F40027A0330690427
:100D2D00781E7A01206007E53D6003D2AF22D2AF75
:100D3D000000C2AFC3E53BFB940F40027B0FEB04F9
:100D4D003073012320620123F93069027982E58B2A
:100D5D00C39940D0053DEAFBE59BF45440B5200412
:100D6D00DBF6A19520650281F9C265759100AE3A59
:100D7D00AF3BC3E49EF594E49FF595759104D26065
:100D8D0053917F43E68081F930650281F9D895D280
:100D9D00AF2230690B0534206016753400020DBD8D
:100DAD0020600D20650A206B07158115810215A5A0
:100DBD0022A84EA94F75910053917FC3E498F594E5
:100DCD00E499F595759104854850854951D2604354
:100DDD00E6802278003064053065027801E53575CE
:100DED00F007A4F9E5F028F5F0E9A2F013A2F1134C
:100DFD00A2F213F535C394785003753578C3E535F4
:100E0D0095364008D266D292D291D290306002C10E
:100E1D0019854A50854B51D26043E68022C2AFC23C
:100E2D0093C294C29530720B9001FF7406D5E0FD0C
:100E3D00020E40207D02D293307D02D295759F1017
:100E4D00753C02020F7FC2AF207D02D290307D0231
:100E5D00D2923072179001DCC294207D02C295307F
:100E6D007D02C2937406D5E0FD020E7C90013F30E9
:100E7D006206E5256002C291207D03759F20307DBD
:100E8D0003759F00753C03020F7FC2AFC293C294DE
:100E9D00C29530720B9001B97406D5E0FD020EAD0E
:100EAD00207D02D295307D02D293207D03759F0067
:100EBD00307D03759F20753C04020F7FC2AFD29128
:100ECD00307217900196207D02C293307D02C2953B
:100EDD00C2947406D5E0FD020EEA90012D30620E2B
:100EED00E525600A207D02C292307D02C290759F79
:100EFD0010753C05020F7FC2AFC293C294C29530EC
:100F0D00720B90016B7406D5E0FD020F1AD294207E
:100F1D007D03759F20307D03759F00753C06020F84
:100F2D007FC2AF207D02D292307D02D29030721FEF
:100F3D0090022A207D02C293307D02C295207D024F
:100F4D00C295307D02C2937406D5E0FD020F5F900D
:100F5D00015130620EE525600A207D02C290307D80
:100F6D0002C292207D03759F00307D03759F207511
:100F7D003C01306B13120F9A7406D5E0FD7406D543
:100F8D00E0FDD293D294D295C266D2AF2290012BBE
:100F9D00D292D291D290C293C294C295C26222785B
:100FAD008076090876090876040876010876030824
:100FBD0076FF087609087601087601087601788CA7
:100FCD0076010876FF0876FF0876FF0876FF08762B
:100FDD00FF0876030876FF0876FF0876FF0876256A
:100FED000876D00876280876500876040876FF082B
:100FFD00760208760008767A0876FF087601227860
:10100D0087E6FFC272BF0302D2727888E6C39403EB
:10101D006008C27DE630E102D27DC27E7889E6307D
:10102D00E102D27EC3EF94026008758E01D2730285
:10103D001044758E00C273227880E6149000809360
:10104D0078A1F67881E6149000809378A2F6120FBD
:10105D009A227886E61490008D9378A3F6120F9A53
:0E106D002222789CE67536FF75370CB4020619
:10107B007536A075370AB4030675368275370522A7
:10108B00227896E6FA7897E6FB307F047A007BFFAE
:10109B00C3EB9AFCC3948250027C82756F00056F80
:1010AB00EC856FF0A4C3E5F0948040F222D27F115F
:1010BB008C1206D57A007B007C101206CBE5592AE0
:1010CB00FA74003BFBDCF37C04C3EB13FBEA13FA6F
:1010DB00DCF7FEC27F118C22E5EF20E603752000C2
:1010EB000520903FFFE520146006901DFF14600063
:1010FB009304600375EF12C2D353D9BF7581C043FC
:10110B00FF801206C675EF0243B203E5B324042039
:10111B00E702F5B3120F9A7580FF75A40075F1D431
:10112B0075D4EF75908775A54075F2FF75D5BF75B2
:10113B00A60175E24275DB4675EA02120FAC121579
:10114B00D678988670C2AF1206DF1206EF1206D55C
:10115B001206F61206D51206FD1206D5C2AFE4F83A
:10116B00F6D8FD78C879C8308407D9FBD8F7021CAC
:10117B0000120FAC1215D6110C1145115F116E1127
:10118B006F118B118C78988670120F9A7588507529
:10119B00891275C82475910475D84075A82275B845
:1011AB000275E690759B80759D0075D10E75BC58C8
:1011BB0075BB0375BA1175E8801206C6D2AF12095A
:1011CB00E643DA01C2D8C2711206DF753001D26173
:1011DB007B037A0CE55870067A0CDB02216712064A
:1011EB00D52070022167C270E559C3940240E3E534
:1011FB002F541F855B5AF55BB55AD7DAD7C26153AB
:10120B00DACF207E0343DA20307E0343DA10C2D8D4
:10121B00C271C2757528001206DA307409C3E5284D
:10122B00940A4002D2751206CB7802307402780011
:10123B00C3E5599840F0C2AF1206EF1206EF120643
:10124B00EFD2AF1206DF7546007888E6B403026171
:10125B00301206CB788CE6C394015003021330E5B1
:10126B0030C394015003021330207435C3E55994F5
:10127B00FF5003021330C2AF120704D2AF1206DACB
:10128B00C3E559940150EFC2AF1206EF1206D0120C
:10129B0006EFD2AF1206DAC3E55994FF40E9021705
:1012AB007E7F02D27F118C1206DAC2AFC27F118C05
:1012BB00AE59C3E559947FD2AF40741206C6C2AF84
:1012CB00120704D2AFDFDC11B8C3EE94057897F6A2
:1012DB001206DF1216181217017F0AD27F118C1219
:1012EB0006DAC2AFC27F118CAE59C3E559947FD2D7
:1012FB00AF50E61206C6C2AF1206EF1206D01206A8
:10130B00EFD2AFDFD611B8EE24057896F61206DFD2
:10131B001216181217301206DA118CC3E55994FF06
:10132B0040F402177EC3E559954640038559461292
:10133B0006DA78017988E7B403027805C3E5599892
:10134B0040024154C2AF120704120704120704D221
:10135B00AF1206DF753000E4F531F5320531E531BA
:10136B00F470390532789AE67819146012783214D1
:10137B00600D787D14600878FA146003753200C331
:10138B00E53298401715327531B478998670C2AF33
:10139B00120704D2AF789886701206DA1206D0E5DF
:1013AB00297005307402216778012074027806C316
:1013BB00E5599840A77888E6C3940360031206DAD0
:1013CB00E52970022167C2AF120F9AE4F522F523CB
:1013DB00F524F525D2AF78858662F53EF53FF540CD
:1013EB00F541F542F56DF547F52CF52DF535120B5D
:1013FB0075756D0875BB101206C6120A81E5E820DB
:10140B00ECFBA8BDA9BEE97001F8886E120A8575C0
:10141B006D0875BB107887E6FE7602110C7887EEA7
:10142B00F6C2AF755EFF120B5785225E85225F8574
:10143B002260D2AF752201752401752501855D648B
:10144B00756501D268D269753400120F04120F2E24
:10145B00120B75120B7C120BF2021472120F9A11F3
:0D146B000C756D0075BB03120CF1120D9F86
:10147800120DBE1207EE120DE0120E2A120B7C128C
:101488000BE1120BF2120CAE120CE6120D9F120DAC
:10149800BE12084C1209AA120DE0120E53120B7C50
:1014A800120BE1120BF2120CAE120CF1120D9F127C
:1014B8000DBE120885120DE0120E97120B7C120B4E
:1014C800E1120BF2120CAE120CE6120D9F120DBEB9
:1014D8001208E2120DE0120EC9120B7C120BE11277
:1014E8000BF2120CAE120CF1120D9F120DBE120966
:1014F80047120DE0120F04120B7C120BE1120BF2D3
:10150800120CAE120CE6120A81120D9F120DBE12B9
:101518000A85120DE0120F2E120B7C120BE1120B32
:10152800F2120CAE306938206B3585615E85615FDB
:10153800855D6475650179327A0AC3E5349940128C
:10154800C269D26A8A3385615E755FFF7560200261
:101558001567C3E559940140030214720215A530BA
:101568006A1E206B1BE533147007C26A755EFF8123
:1015780067F533C3E559940140030214720215A5B7
:10158800C3E55C94FA5016307404E529600FC3E58E
:101598003B78F0306B0278609850028172C2AF12CB
:1015A8000F9A7887E6FE7602110C7887EEF6E4F556
:1015B80022F523F524F525F562C268D2AF1206C6D6
:1015C800120F9A307406E529700221676162901A39
:1015D8000D782012165AE520B4550CA312165AE5B8
:1015E80020B4AA030215F8120FAC12161802161727
:1015F800901A0378807B0A12165AA308DBF9901A0E
:101608000F788C7B1512165AA308DBF9901A24223E
:10161800C2AF121699121673901A00740D12165F43
:10162800A3740212165FA3741312165F901A03783C
:10163800807B0A12165EA308DBF9901A0F788C7B60
:101648001512165EA308DBF91216AC12168A901A48
:101658002422E493F622E6438F01538FFD75EF02AF
:1016680075B7A575B7F1F0538FFE22438F02438FEC
:101678000175EF0275B7A575B7F1901A0DF0538F84
:10168800FC22901A0D7455D15F901A0E74AAD15F7E
:10169800227A3079D07820901A40D15AE520F7097B
:1016A800A3DAF7227A3079D0901A40E7D15F09A3FC
:1016B800DAF922AB71A872BB01027980BB02027908
:1016C80081BB03027982BB04027984BB050279835A
:1016D800BB06027986BB07027992BB08027987BBF1
:1016E8000902799CBB0A027988BB0B027989E8F761
:1016F800227C051206DFDCFB22C2AF1206EF1206BF
:10170800F61206FD1207041206D01206EF1206F6AC
:101718001206FD1207041206D01206EF1206F61280
:1017280006FD120704D2AF22C2AF1207041206FD4B
:101738001206F61206EF1206D01207041206FD1260
:1017480006F61206EF1206D01207041206FD12065C
:10175800F61206EFD2AF22AE71AF72C2AF1206EF29
:101768001206EF1206EF1206D0DEF2120704120676
:10177800D0DFF8D2AF22F101D1F9D1F97571017535
:101788007201757300F15F7C05AD591206DFC3ED78
:10179800955970F5C3E5599401400AC3E55994FF7A
:1017A80040320217BAD1BBD118F101C2AF75EF129E
:1017B800D1F9DCD50573C3E5739403500280C6D113
:1017C800F90572E5711490009A93F808C3E57298C8
:1017D800500280AED1F9D1F90571C3E571940C506E
:0F17E80002809C120FACD118C2AF75EF12D1F96D
:101A00000D02130909040103FF0901010155AA018F
:101A1000FFFFFFFFFF03FFFFFF25D0285004FF0259
:051A2000007AFF01FF48
:101A400023484B696E673530412320202020202019
:101A500023424C48454C4923463333302320202031
:101A60002020202020202020202020202020202076
:101C0000C2AFC2D353D9BF7581C043B20343FF8073
:101C1000752438752503B1BF75EF0275E24043F1B5
:101C20001053A4EFD284780379E67C1075220075F6
:101C30002300901DCC7B0675249875250130840205
:101C4000813D208408D8FBD9F9DCF781AD308408C8
:101C5000D8FBD9F9DCF781ADB17FE493A3C39A60D7
:101C6000028126DBDDB171600281267B08E493FAF4
:101C7000A3B152DBF87A30B152752200752300B15E
:101C800071EAFCEBFDC3ED94FE400EB1718A278B27
:101C900028ED30E0048A828B83B1717AC270D8C398
:101CA000ED94FE601050CEBD0022EC600675200061
:101CB0000200008100A827A9280809D804D90281B8
:101CC000C9B175EA89AAF281BB0D8199C3ED94036C
:101CD0005049EDA2E092007AC5C3E5829400E58305
:101CE000941C5093200010438F02438F0175B7A5B9
:101CF00075B7F1F030001FA827A9280809438F0104
:101D0000538FFDD804D902A11689AAE275B7A5752B
:101D1000B7F1F0A3A103538FFC81757AC1BD030C09
:101D2000E493A3FAB136DCF8B12E81758177AA224B
:101D3000AB23B152EBFAEA6222752608C3E52313FE
:101D4000F523E52213F52250066323A0632201D573
:101D500026EAB1BFB1BF75260AEAF4200102D28497
:101D6000300102C284B1BFC3134002C201D526EBC9
:101D700022B175EAFB208402A175308402A17A7534
:101D80002608AE24AF25C3EF13FFEE13FEB1C3B197
:101D9000BFC3EA133084024480FA30E703632201B0
:101DA000C3E52313F523E52213F52250066323A090
:101DB000632201D526D9E52265236523F52222AECB
:101DC00024AF250E0FDEFEDFFCD20122424C486517
:0A1DD0006C6934373132F33006013C
:00000001FF
